:100000000EC013C012C011C010C00FC00EC00DC072
:100010000CC00BC00AC009C008C007C006C011242C
:100020001FBECFEDCDBF29D062C0EACF20ED37E0B3
:1000300003C0F9013197F1F70197D8F70895A39A12
:1000400083EA87B986EC86B93699FECF369A369917
:10005000FECF85B1089585E088BD85E090E0E6DFBC
:1000600018BC88EC90E0E2CF84E188BD86E990E09E
:10007000DDDF18BC88EC90E0D9CF82E087BB81E25D
:100080008ABD81E083BF81EA87B9A29A86EC86B9EE
:10009000479AD5DFE82EF12C3798BB9AC39A00E037
:1000A00010E003C0E1DF04561109E801CE0DDF1DA9
:1000B000C436D105B8F788EE93E0B8DFCA30D10571
:1000C00020F4C9DF02C02A97CFDFCA30D105D8F7A4
:1000D00088EE93E0ABDF209721F4BDDF02C02197CB
:1000E000C3DF2097E1F788EE93E0A0DFFCCFF89420
:0200F000FFCF40
:00000001FF
